S123E0000F8604973F8608972686409724860297098620972B862C972D962F7F004B8E009E
S123E020FF0ECE08E0C60218CE0019BDE03ABDE06020FBDF49DE4926FC3918DF43BDE1D809
S123E04018DE4318DF4718DE4726FB7F00227F002018DE4318DF4718DE4726FB5A26DE393B
S123E060964B81FF27037EE0E87F004BBDE1B096408141272E8161272A8143273781632766
S123E080338144273D8164273981532746817327428134250981362205BDE0E9204ABDE1EE
S123E0A0022045CEE308BDE1CBD6004FBDE16DBDE1B02034CEE316BDE1CB7F0000BDE1B004
S123E0C02026CEE30FBDE1CBD6084FBDE16DBDE1B02015CEE32CBDE1CBBDE1B0CE08E0C602
S123E0E00218CE0019BDE03A39C6018030584A26FCD5002703532005DA00D70039D400D7C4
S123E1000039BDE1BBCEE2DBBDE1CBBDE1B0CEE2AEBDE1CBBDE1B0CEE2DBBDE1CBBDE1B0D0
S123E120CEE210BDE1CBBDE1B0CEE229BDE1CBBDE1B0CEE244BDE1CBBDE1B0CEE25DBDE17E
S123E140CBBDE1B0CEE281BDE1CBBDE1BBCEE2ACBDE1CB394FCE0064028FD7418FCE000A20
S123E16002D7428F58585858DA42D742394FBDE15496418B30BDE1A99642BDE17E39368422
S123E180F044444444810A2D06800A8B4120028B30BDE1A93236840F810A2D06800A8B4134
S123E1A020028B30BDE1A93239D62E2AFC972F39860DBDE1A9860ABDE1A939860DBDE1A9DF
S123E1C0860ABDE1A9860ABDE1A939A60081FF2706BDE1A90820F4390FDF4586409720971E
S123E1E02397220E39DE47270309DF47DE49270309DF49864097253B962E962F974086FF56
S123E200974B3BDC45D318DD18CE00001D23BF3B4120203D3E2053484F5720504F525420F2
S123E2204120535441545553FF4320203D3E20434C45415220504F52542041204F555450E3
S123E240555453FF4420203D3E2053484F5720504F5254204420535441545553FF53202000
S123E2603D3E204245455020535045414B45522028434F4E4E45435420544F205041362993
S123E280FF3420544F2036203D3E20544F47474C45205448452053454C45435445442050D7
S123E2A04F525441204F5554505554FF3FFF39204D487A204D4943524F5354414D503131ED
S123E2C02044454D4F2050524F4752414D20434F4D4D414E44204D454E55FF5F5F5F5F5F6F
S123E2E05F5F5F5F5F5F5F5F5F5F5F5F5F5F5F5F5F5F5F5F5F5F5F5F5F5F5F5F5F5F5F5F3A
S123E3005F5F5F5F5F5F5FFF504F5254413DFF504F5254443DFF504F525441204F555450EC
S11DE32055545320434C4541524544FF3E3E3E204245455021203C3C3CFFEA
S123FFD6E1F8E000E000E000E000E000E000E000E203E000E000E000E000E1E5E000E00023
S10DFFF6E000E000E000E000E0009D
S9030000FC
